:10000000789D001001010000090100000B010000B3
:100010000D0100000F01000011010000465CFFEF20
:1000200000000000000000000000000013010000BC
:10003000150100000000000017010000A5360000B7
:100040001B010000E93800001B0100001B0100003B
:100050001B0100001B0100001B0100001B01000030
:100060001B0100001B0100001B0100001B01000020
:100070001B010000000000001B0100001B0100002C
:100080001B0100001B0100001B0100001B01000000
:100090001B0100001B0100001B0100001B010000F0
:1000A0007D3C00001B0100001B0100001B01000043
:1000B0001B0100001B0100001B0100001B010000D0
:1000C0001B0100001B0100001B0100001B010000C0
:1000D0001B0100001B0100001B0100001B010000B0
:1000E0001B010000DFF80CD000F05EF8004800476C
:1000F000ED480000789D0010D0F800D0D0F804F052
:100100000648804706480047FEE7FEE7FEE7FEE7B1
:10011000FEE7FEE7FEE7FEE7FEE7FEE74138000008
:10012000E500000010B50B4604461146184600F0E5
:1001300027F8C4E9000110BD40EA01039B0703D082
:1001400009E008C9121F08C0042AFAD203E011F816
:10015000013B00F8013B521EF9D27047D2B201E0D8
:1001600000F8012B491EFBD270470022F6E710B5BC
:1001700013460A4604461946FFF7F0FF204610BD15
:1001800070B500242546002801DA012440420029E8
:1001900001DA0125494200F019F8AC4200D0404292
:1001A000002C00D0494270BD064C074D06E0E068C7
:1001B00040F0010394E8070098471034AC42F6D3AE
:1001C000FFF794FF145400003454000030B50B4680
:1001D000014600202022012409E021FA02F59D4277
:1001E00005D303FA02F5491B04FA02F52844151E4B
:1001F000A2F10102F1DC30BD30B58C1810F8012BF2
:1002000012F00F0301D110F8013B120906D110F8CA
:10021000012B03E010F8015B01F8015B5B1EF9D1D3
:1002200001E001F8013B521EFBD1A142E6D30020C0
:1002300030BD00000B4880680B490A68801A4A6884
:1002400002EB4203C3EBC212B0EBC20F08D3074864
:1002500002224260C26B02F0FE02C26300204860CC
:100260007047000000000940F000001000800040CE
:10027000074800210167C16002224261816130228A
:10028000C263044882680448C0E9002108467047F8
:100290000080004000000940F000001070B50D4CD7
:1002A00000250E46656000F02BF80B4A06EB460170
:1002B0002068C1EBC61193681B1AB3EBC10FFAD3C8
:1002C000064802214160C16B01F0FE01C1630020BC
:1002D000656070BDF0000010000009400080004023
:1002E0000020704701460007C00E090600D5401CDB
:1002F0007047002070474FF480507047FFFFFFFFAA
:1003000070B541F28832904215D8642800D290B975
:1003100042F2107291420ED805290CD30F4CA268FC
:100320000F4B1D68521B5D6805EB4506C6EBC515F6
:10033000B2EBC50F01D2002070BD0A4A02255560FC
:1003400038B1094EB6FBF0F04010906155600120C5
:100350005060A068C3E90001EDE70000000009401B
:10036000F00000100080004080C3C90170B5002378
:10037000084D0AE0CE5C04885B1C86EA14269BB21A
:1003800035F8166086EA04240480521E92B2F1D237
:1003900070BD0000284E00002DE9FC4107460020FA
:1003A00090460E46ADF8000004460EE0351B402D89
:1003B00000D9402539192A460D4800F00CFCAAB294
:1003C0000B496846FFF7D2FF2C44B442EED33919EB
:1003D000424601A800F0FFFBBDF80000BDF8041084
:1003E000884202D10120BDE8FC810020FBE700002B
:1003F0003801001001480068704700002401001017
:10040000704770474D0B00002DE9F041664C002706
:1004100088B0A770E770DFF894814FF40056277119
:1004200001251922314601A800F0D5FB0222162130
:100430003046FFF7B1FF00287ED0DDF8121002220F
:1004400006F11900FFF7A8FF002875D09DF80400F9
:1004500006282AD2DFE800F02A03032A2A1CD8F84B
:100460007410DDF80E30491C8B421ED2D8F874206F
:10047000DDF80E30D21ADDF81230521C9A4214D335
:10048000DDF80E20DDF812301A448A420DD80DE056
:10049000DDF81210B1F5F42F00D9A570DDF81610B3
:1004A000C1F30B41B1F5B07F00D0A570012803D096
:1004B000022801D0052839D1022206F21D416846E2
:1004C000009700F088FB0099029889B2884200D01A
:1004D000A570012206F225416846009700F07BFBDB
:1004E0000099BDF80500C9B2884200D0A5709DF8FA
:1004F000040002281AD1042206F2494168460097F6
:1005000000F069FBDDF816000099884200D0A57064
:10051000012206F24D416846009700F05CFB00980E
:100520009DF80710C0B2814200D0A5709DF81C0054
:10053000401EFE2802D200E01EE0A570BDF80500B6
:10054000A0F57F41FF3901D0402802D19DF8070076
:1005500020B901A800F042FA00B9A570DDF8120038
:100560001B36064401A800F039FA30B1E07880B1BA
:10057000217988420DD012E0A5709DF81C0010B9B9
:100580002079401C2071E078401CC0B2E0700C283B
:1005900001D3A57003E0A07800283FF442AFA07813
:1005A00008B0BDE8F08100000C000010E051000030
:1005B00070B500F049F81049104D114E114C0870FB
:1005C00050B1114900EBC00001EB8000806880470A
:1005D000000609D5206870BD822020602120286097
:1005E00078463060822070BD002020602860784608
:1005F0003060002070BD00002C010010840000104D
:1006000088000010800000103C530000094800786A
:1006100028B1094900EBC00051F820000047074904
:100620008220086006492120086078460549086054
:10063000822070472C0100103C5300008000001005
:10064000840000108800001070B5002400BF00BFB7
:1006500000BF00BF00BF00BF00BF00BF00BF00BFA2
:1006600000BF00BF00BF00BF00BF00BF00BF00BF92
:1006700000BF00BF00BF00BF00BF00BF00BF00BF82
:1006800000BF00BF00BF00BF00BF00BF40252D4E10
:10069000F5619F2001F02AFC002001F027FC60F3A7
:1006A0000704002001F022FC60F30F24002001F079
:1006B0001DFC60F31744B56100BF00BF00BF00BF61
:1006C00000BF00BF00BF00BF00BF00BF00BF00BF32
:1006D00000BF00BF00BF00BF00BF00BF00BF00BF22
:1006E00000BF00BF00BF00BF00BF00BF00BF00BF12
:1006F00000BF00BF00BF00BF1349601A8C421AD070
:100700000BDCA4F1C204B4F5A11414D0B4F5803FFD
:1007100011D0B4F5003F0BD10DE00C49401805D0C5
:100720000B49401809D00B49C84201D1022400E00E
:100730000024204670BD0324FBE7042402F076FC6D
:10074000F7E7000000800920C220180003FBD6FF55
:1007500000FFFEFF0001F8FF0549822008600549FF
:100760002220086078460449086082207047000013
:1007700080000010840000108800001005498220CD
:1007800008600549212008607846044908608220F5
:1007900070470000800000108400001088000010E6
:1007A00005498220086005492220086078460449EE
:1007B0000860822070470000800000108400001054
:1007C000880000102DE9F041144B154D154E1B7893
:1007D000154C63B19AB1154F03EBC30307EB8303C9
:1007E0001B699847000612D52068BDE8F081822079
:1007F000206021202860784630608220F5E786203E
:10080000206009202860784630608620EDE70020CF
:1008100020602860784630600020E6E72C01001058
:100820008400001088000010800000103C5300007D
:100830002DE9F041144B154D154E1B78154C63B145
:100840009AB1154F03EBC30307EB83039B699847EA
:10085000000612D52068BDE8F081822020602220A9
:100860002860784630608220F5E7862020600920E5
:100870002860784630608620EDE700202060286000
:10088000784630600020E6E72C010010840000105C
:1008900088000010800000103C530000F8B5184C90
:1008A000184D194E2778194CDDF818C087B1BCF1E6
:1008B000000F15D0CDF800C0DFF854C007EBC70714
:1008C0000CEB8707FF69B847000611D52068F8BD13
:1008D0008220206022202860784630608220F8BD87
:1008E0008620206009202860784630608620F8BD88
:1008F000002020602860784630600020F8BD0000AD
:100900002C010010840000108800001080000010EE
:100910003C53000070B50948022400F11F058168AE
:1009200029B1007B000607D4022003F081FC2C7360
:1009300000F016FC002070BD012070BDD11B00101E
:1009400010B50C480C4C8068A178884200D2A07089
:100950000849A2784039822003F09AFC0320607095
:100960000448A2781F308168891A816000210173D0
:1009700010BD0000D11B00108C0000102DE9F041CB
:10098000092000F051F8124800264FF47A770670DB
:10099000C8213846FFF782FC0E4CA06842F2107561
:1009A000A168091AA942FBD3C8213846FFF776FC93
:1009B000A068A168091AA942FBD3C8213846FFF7ED
:1009C0006DFC0548022186708171C670BDE8F0811A
:1009D0007C000010000009400C0000100021425C67
:1009E00012B9491C1829FAD3182901D000207047E0
:1009F00001207047014600200A4A4B0703D5536F78
:100A00009B0100D50420CB0704D0536FDB0101D537
:100A100040F00100890704D5516F490101D540F02C
:100A2000020070470080092070B54F4B50B15968E3
:100A3000042403250226052907D2DFE801F0072D4B
:100A40004C74910000205860986070BD042807D055
:100A5000052809D0012402287DD0012809D011E001
:100A6000072000F083F848E0BDE87040012000F066
:100A70007DB8072000F07AF80CE000BF00F08AF89B
:100A80005C6070BD0E28FCD1072000F06FF80220DA
:100A900000F080F80120F1E706280AD0032810D0E2
:100AA0000A2813D0092811D00D280FD00C28D7D030
:100AB00070BD072000F05AF8022000F06BF85E606D
:100AC00070BD072000F052F8012028E0072000F058
:100AD0004DF8022012E0062814D00A281BD009285D
:100AE000C7D00C28BCD00D28F0D00F28E8D10720A3
:100AF00000F03CF8022000F04DF80120BDE8704005
:100B000000F048B8986810F01F0F00F101009860DD
:100B1000D6D102201BE0072000F028F8022000F0C8
:100B200039F85D6070BD072806D00A2898D00B28D8
:100B300011D009289DD070BD022000F017F89868E8
:100B400010F03F0F00F101009860F4D10120BDE8E2
:100B5000704000F033B8072000F008F802208DE75D
:100B60000628A6D08EE70000D000001008494207F2
:100B700002D54FF00072CA67C20702D04FF08072F0
:100B8000CA67800702D54FF08060C86700207047B1
:100B9000008009200849420702D54FF000728A6799
:100BA000C20702D04FF080728A67800702D54FF0EB
:100BB00080608867002070470080092010B50446D7
:100BC000FFF718FF0346FFF7D1FF24EA0300FFF702
:100BD000E1FF002010BD10B50B4601460024184669
:100BE000FFF7F0FD204610BD0E4810B541780229F0
:100BF00008D003290ED0042910D0052901D10021E5
:100C0000417010BD0848C07B2828FAD1BDE81040CB
:100C100000F034B9BDE8104000F0A2BA822003F021
:100C200007FBF7E78C000010D11B001010B514492A
:100C3000022003F007F913498870487860B1012851
:100C40000ED0022003F0F4FA0D4902205F31087340
:100C5000BDE8104000F084BABDE8104000F014B8C0
:100C600007484030C07B2A2805D02F2807D1BDE88F
:100C7000104000F035B9BDE8104000F075B910BD66
:100C8000911B00108C0000102DE9F0414A4D4B4C97
:100C90000021A878A4F1400202E0535C6354491C8F
:100CA00003468142F9D31F2B7CD1206844498842F6
:100CB00078D1424E60681F364FF001087060A0681E
:100CC000B060607B18B9A07B08B1102802D986F803
:100CD0000C8063E0E07B1E28F9D011DC122833D0B1
:100CE00006DC68B30328F2D1BDE8F04100F00EBA8B
:100CF0001528ECD01A28EAD1BDE8F04100F07EB901
:100D000002272A282ED011DC232821D0252823D001
:100D10002828DCD100F08AF900282CD0207B00069E
:100D20001ED56F70BDE8F04100F0A8B82F2824D080
:100D30005528CCD05A28CAD1BDE8F04100F042B9BC
:100D4000BDE8F04100F01EBABDE8F04100F03AB84D
:100D5000BDE8F04100F0B4B9BDE8F04100F08EB953
:100D6000022018E000F062F9002804D0207B000681
:100D700010D485F80180BDE8F08100F057F9002813
:100D8000F9D0207B000605D485F80180C5F82880BD
:100D9000F1E707E0822003F04BFA3773BDE8F0413A
:100DA00000F0DEB9822003F043FA022003F040FA9B
:100DB00006206870DFE700008C000010D11B0010D7
:100DC000555342431CB5FFF7A5FD00284ED02848D7
:100DD0000A2206210388684603F024FF25480022E2
:100DE00080230270437082700121C1702021017143
:100DF00043718271C27141220272542242724F22A7
:100E000082724C22C272017341738173C173462294
:100E1000027450234374722383746923C3746E2352
:100E20000375742343758175C2756C220276612245
:100E30004276732282766822C27601774177817783
:100E4000C1779DF8011080F820109DF8021080F8FD
:100E500021109DF8031080F822109DF8041080F8EE
:100E60002310054924208870FFF76AFD1CBD00008F
:100E700004040000911B00108C00001070B5154D8B
:100E80002C6B402C00D94024E86AE96902198A4297
:100E900002D90C1A04216970214603F00FFE224684
:100EA0000D49822003F0F4F9E86A2044E862286BD7
:100EB000011B0A4829638268A2EB0402826005D004
:100EC0006978022901D00021017370BD0321697086
:100ED000F9E700008C00001038010010F01B001032
:100EE0002DE9F0411D4CA178E06A4218E1698A427F
:100EF00006D9081AA07005206070022003F098F946
:100F00000021A078164B174DE26A08E056186F5C76
:100F10009E5DBE4202D00021A16202E0491C8142D6
:100F2000F4D31118E162216B0A1A0E49226301F110
:100F30005F018B68A3EB0000886002D06078052811
:100F400009D1A06A28B100200873BDE8F04100F083
:100F500007B90120F8E7BDE8F08100008C0000101F
:100F600038010010911B001010B5144CA178E06AF4
:100F70004218E1698A4206D9081AA07005206070FB
:100F8000022003F055F9A178E06A03F0DDFDA178B5
:100F9000E06A0844E062206B421A094822638368D1
:100FA000A3EB0101816002D06178052905D1002100
:100FB0000173BDE8104000F0D3B810BD8C000010E4
:100FC000F01B001010B5FFF7A5FC002811D0094850
:100FD00000210622017042708170C170017141715F
:100FE0008171C171044908208870BDE81040FFF785
:100FF000A7BC10BD911B00108C00001010B5FFF7AE
:1010000089FC00280DD007480321017000214170A0
:101010008170C170044904208870BDE81040FFF75A
:101020008FBC10BD911B00108C000010114810B532
:10103000D0F81110027D09BA21F0FF0111430E4AC8
:101040004902D162C18A49BA490211638068884263
:101050000DD0822003F0ECF8022003F0E9F80549F6
:1010600002201F31087300F07BF8002010BD012022
:1010700010BD0000D11B00108C00001010B5FFF750
:1010800049FC002816D00C4A0C48116A491E0B0E68
:1010900003700B0C43700B0A8370C1700021017147
:1010A000417102238371C17108209070BDE8104026
:1010B000FFF746BC10BD00008C000010911B001013
:1010C00010B5FFF727FC00281AD00E4800210E4B60
:1010D0000170417081700822C2701A6A140E047186
:1010E000140C4471140A8471C2710222027241729A
:1010F0008272C1720C209870BDE81040FFF720BCCE
:1011000010BD0000911B00108C00001010B5FFF7FF
:1011100001FC00281FD0104870210222017000211C
:1011200041708270C1700171417181710A22C27176
:10113000017241728172C1723022027301224273C4
:101140008173C17301744174044912208870BDE831
:101150001040FFF7F5BB10BD911B00108C00001074
:10116000064910B5044808600D22822003F090F86B
:1011700003490520487010BD55534253F01B001021
:101180008C000010094810B5816839B1007B000659
:1011900001D5822000E0022003F04AF80349002034
:1011A0001F310873BDE81040FFF7DABFD11B0010F4
:1011B0002DE9FC5F8846044601A9414800F0B8FAD1
:1011C000404D414E414FE0BB03208DF80000200907
:1011D0008DF8010020018DF802004FF000098DF814
:1011E000039000BF00BF00BF00BF00BF00BF00BF33
:1011F00000BF00BF00BF00BF00BF00BF00BF00BFF7
:1012000000BF00BF00BF00BF00BF00BF00BF00BFE6
:1012100000BF00BF00BF00BF00BF00BF00BF00BFD6
:1012200000BFDFF8ACB04FF0400ACBF81CA004219F
:10123000684600F065FE0024002000F057FEC0B2B2
:1012400000E005E08DF8040018F80410884208D08A
:101250008220286022203060784638608220BDE8F5
:10126000FC9F641CB4F5805FE6D3CBF818A000BFE8
:1012700000BF00BF00BF00BF00BF00BF00BF00BF76
:1012800000BF00BF00BF00BF00BF00BF00BF00BF66
:1012900000BF00BF00BF00BF00BF00BF00BF00BF56
:1012A00000BF00BF00BF00BF00BF00BF00BFC5F848
:1012B00000907846C6F8009038600020CFE7000024
:1012C000A08601008000001084000010880000103B
:1012D000008009202DE9F0474FF0000900BF00BF52
:1012E00000BF00BF00BF00BF00BF00BF00BF00BF06
:1012F00000BF00BF00BF00BF00BF00BF00BF00BFF6
:1013000000BF00BF00BF00BF00BF00BF00BF00BFE5
:1013100000BF00BF00BF00BF00BF00BF4025334E6D
:10132000F5619F2000F0E2FD002000F0DFFD00F0FD
:10133000FF08002000F0DAFDC4B2002000F0D6FD66
:10134000C1B2B56100BF00BF00BF00BF00BF00BF9A
:1013500000BF00BF00BF00BF00BF00BF00BF00BF95
:1013600000BF00BF00BF00BF00BF00BF00BF00BF85
:1013700000BF00BF00BF00BF00BF00BF00BF00BF75
:1013800000BF00BF1A4D1B4E1B4FB8F1C20F01D159
:10139000202C08D0822028602120306078463860D8
:1013A0008220BDE8F0871548142912D0152913D0E2
:1013B000162915D0182916D0C0F80090002000F08A
:1013C000C7F8C5F800907846C6F80090386000204D
:1013D000E7E74FF4801101E04FF400110160EDE701
:1013E0004FF48001FAE74FF08071F7E700800920A1
:1013F00080000010840000108800001024010010FC
:101400002DE9F04FDFF89480DFF894B089B00F0039
:1014100004464FF0000628D04FF4805501462A4676
:101420006846FEF77FFEDDE900A105912A462146C8
:1014300006A8FEF777FEDDE906404FF00009BD1B68
:10144000C0F58051A94200D20D4620B1544517D1B4
:101450000599884214D1204600F0C4FE00060FD53D
:10146000D8F8000009B0BDE8F08F8621C8F8001058
:101470000921CBF8001079460A4801608620F1E77F
:101480002E44641C4846BE42D9D3C8F800007946B1
:10149000CBF80000034801600020E3E78000001063
:1014A000840000108800001070B5044600BF00BF23
:1014B00000BF00BF00BF00BF00BF00BF00BF00BF34
:1014C00000BF00BF00BF00BF00BF00BF00BF00BF24
:1014D00000BF00BF00BF00BF00BF00BF00BF00BF14
:1014E00000BF00BF00BF00BF00BF00BF4025174EB8
:1014F000F561052000F0FAFC002000F0F7FC2070F8
:10150000B56100BF00BF00BF00BF00BF00BF00BF8C
:1015100000BF00BF00BF00BF00BF00BF00BF00BFD3
:1015200000BF00BF00BF00BF00BF00BF00BF00BFC3
:1015300000BF00BF00BF00BF00BF00BF00BF00BFB3
:1015400000BF207800F0010070BD0000008009207D
:101550002DE9F047744E80464FF080773068402484
:10156000724DB84249D100BF00BF00BF00BF00BFED
:1015700000BF00BF00BF00BF00BF00BF00BF00BF73
:1015800000BF00BF00BF00BF00BF00BF00BF00BF63
:1015900000BF00BF00BF00BF00BF00BF00BF00BF53
:1015A00000BF00BF00BFEC61152000F09FFC0020D1
:1015B00000F09CFC00F0FF09AC6100BF00BF00BF61
:1015C00000BF00BF00BF00BF00BF00BF00BF00BF23
:1015D00000BF00BF00BF00BF00BF00BF00BF00BF13
:1015E00000BF00BF00BF00BF00BF00BF00BF00BF03
:1015F00000BF00BF00BF00BF00BF00BF00BF00BFF3
:1016000000BF00BF00BF00BF00BF00BF00BF00BFE2
:1016100000BF00BF00BF00BF00BF00BF00BF00BFD2
:1016200000BF00BF00BF00BF00BF00BF00BF00BFC2
:1016300000BF00BF00BF00BF00BFEC61062000F08C
:1016400055FCAC6100BF00BF00BF00BF00BF00BFC2
:1016500000BF00BF00BF00BF00BF00BF00BF00BF92
:1016600000BF00BF00BF00BF00BF00BF00BF00BF82
:1016700000BF00BF00BF00BF00BF00BF00BF00BF72
:1016800000BF00BF00BF00BF00BF00BF00BF00BF62
:1016900000BF00BF00BF00BF00BF00BF00BF00BF52
:1016A00000BF00BF00BF00BF00BF00BF00BF00BF42
:1016B00000BF00BF00BF00BF00BF00BF00BF00BF32
:1016C00000BF00BFEC61012000F010FC4FEA880071
:1016D00000F00CFC3068B84202D1484600F006FC2D
:1016E000AC6100BF00BF00BF00BF00BF00BF00BFB4
:1016F00000BF00BF00BF00BF00BF00BF00BF00BFF2
:1017000000BF00BF00BF00BF00BF00BF00BF00BFE1
:1017100000BF00BF00BF00BF00BF00BF00BF00BFD1
:1017200000BFBDE8F0870000240100100080092000
:101730002DE9F041084C0F460646A56806E0A06872
:10174000401BB04202D30120BDE8F0813846FFF7CC
:10175000ABFE0028F3D1F7E7000009402DE9F04F78
:1017600089B0DFF8F0805FEA020B4FF000060791C6
:101770000FD04FF4805501462A466846FEF7D2FC4A
:10178000DDE90047284603F025F95FEA00090DD09E
:1017900017E086213048C8F8001009210160794619
:1017A0002E480160862009B0BDE8F08F82212A48CA
:1017B000C8F8001022210160794628480160822083
:1017C000F1E7ABEB0605C7F580504FF0000AA842E1
:1017D00000D20546B5F5805F04D02046494600F0AA
:1017E000DFFED8B907982A46811907EB0900FEF7F2
:1017F000A3FC204600F0F6FC80B92046494600F0E4
:101800000DF958B920464946FFF7D2FC78B10AF1E4
:10181000010000F0FF0ABAF1030F05D3484603F0B8
:1018200029F8D8F80000BEE7BAF1000FE1D12E4444
:101830000027641C5E45C4D3484603F01BF80649E4
:101840000020C8F8000008607946044801600020C4
:10185000A9E700008000001084000010880000103C
:101860002DE9FF4F8DB00D46DDF868900026684CDD
:1018700007935FEA09013ED04FF4805701463A468C
:101880006846FEF74FFCDDE900B10C913A46691C51
:101890006846FEF747FCDDE90010CDE904013A4651
:1018A00068460F99FEF73EFCDDE90085A9EB0607C7
:1018B000C5F58050B84200D2074625B1D8457DD144
:1018C0000C9885427AD14FF4805003F083F85FEA98
:1018D000000A1CD0D84550D10C9885424DD12A46DB
:1018E0004FEA0830514600F0D3FD000619D55046A6
:1018F00002F0C0FF7AE0862020604648092101609E
:10190000784645490860862011B0BDE8F08F8220F6
:10191000206040482221016079463F4801608220D2
:10192000F2E70598804509D1049901EB0030C1F533
:101930008052514400F0ACFD0006D8D4404600F07F
:1019400051FC0006D3D407983A46811905EB0A00EA
:10195000FEF7F2FBEA194FEA0830514601F0D2FCDB
:101960000006C4D40599884533D1049800EB0130B2
:101970000499C1F58052514427E0059988450AD160
:10198000049800EB01300499C1F58052514600F0F3
:101990007FFD0006ABD4404600F024FC0006A6D430
:1019A00007983A4681190F98304401F0ABFC0006C5
:1019B0009DD4059988450CD1049800E00DE000EB1A
:1019C00001300499C1F58052514601F09BFC00069C
:1019D0008DD4504602F04EFF0AE007983A4681192E
:1019E0000F98304401F08EFC000601D520688BE78B
:1019F0003E44002508F101084E45FFF457AF054964
:101A000000202060086078460349086000207BE7DA
:101A10008000001084000010880000102DE9F34FB2
:101A20000024474D474E484FC3B080464FF0820ACE
:101A30004FF0210BA14641A94448FFF779FE002849
:101A40006AD101F033F802208DF800004FEA181037
:101A50008DF8010004EB08108DF8020044988DF811
:101A6000039000EB04214FF4807201A8FEF764FBA1
:101A700000BF00BF00BF00BF00BF00BF00BF00BF6E
:101A800000BF00BF00BF00BF00BF00BF00BF00BF5E
:101A900000BF00BF00BF00BF00BF00BF00BF00BF4E
:101AA00000BF00BF00BF00BF00BF00BF00BF00BF3E
:101AB00040202749C8614FF48271684600F020FA3F
:101AC00023494020886100BF00BF00BF00BF00BFA6
:101AD00000BF00BF00BF00BF00BF00BF00BF00BF0E
:101AE00000BF00BF00BF00BF00BF00BF00BF00BFFE
:101AF00000BF00BF00BF00BF00BF00BF00BF00BFEE
:101B000000BF00BF00BF641CE4B2102C93D341A9F6
:101B10000E48FFF70DFE48B1C5F800A07846C6F89C
:101B200000B03860822045B0BDE8F08F00F072FF51
:101B3000C5F800907846C6F8009038600020F2E7BB
:101B4000800000108400001088000010A0860100B2
:101B500000800920C906090E002806DA00F00F00EF
:101B600000F1E02080F8141D704700F1E02080F8BB
:101B700000147047F0B5B649032008630020C1F88F
:101B80000801B44804228265026C42F00402026437
:101B9000B14A8A6600220A611022C261026822F0FC
:101BA000100202600322C1F87022C1F874220022E0
:101BB0004A644FF400328261026842F400320260EB
:101BC0000922C1F80021C1F804211022C1F8D42053
:101BD00052048263026A42F4001202620D22C1F8CA
:101BE000D020C1F8E0200022C1F8F4204FF00052CC
:101BF000C263026A42F0005202620022C1F8F02081
:101C00004FF08052C263026A42F080520262102298
:101C1000CA6702048261026842F000420260102238
:101C2000C1F8142120278765026C42F0200202646B
:101C30001022C1F81C218022C265026C22F08002B1
:101C400002649026C1F8FC600204C263026A22F0BA
:101C5000004202621022C1F808210422C265026C0F
:101C600022F0040202641022C1F8DC20D204C26314
:101C7000026A22F40002026201230B66CB654B6606
:101C80000322C1F8D8200522C1F8E4208B6011227C
:101C9000CA60CB630A640224C1F820411225C1F84E
:101CA00024510C604D600C604D6010248C659C05C7
:101CB000C461046844F4800404600124CC630A64B1
:101CC0001022C1F82C21CA14C265026C42F40062D1
:101CD00002641022C1F830218A14C265026C42F4F9
:101CE0008052026440F282224A629A240C62CA61E3
:101CF00010224A618761026842F0200202601022CD
:101D00008A6140248461026842F04002026001223C
:101D10000A67CA6640F20242CA628A621022C1F8A9
:101D2000E82092058263056A45F08065056210250A
:101D3000C1F8EC505500C563056A25F000650562E1
:101D40004E635513C561056825F4005505600025EF
:101D5000C1F8E851C267026E42F080620266C1F8C3
:101D6000E0511A06C267026E42F080720266C1F844
:101D7000E4515A06C267026E42F0007202668A227D
:101D8000C1F8F8200822C1F8C820D503C563066A47
:101D900046F4802606621026C1F828610E15C66535
:101DA000066C26F4806606640126C1F88060C1F8DE
:101DB0008460C1F89060C1F8A060C1F8A460C1F867
:101DC000A860C1F8B860C1F8BC60C1F8C060C1F8D3
:101DD000C4600026C1F81861C465046C44F0400476
:101DE00004640A655404C461046824F48014046023
:101DF000CA641404C461046824F4002404608A647E
:101E0000C561046824F4802404600024C1F80C41F6
:101E10008265026C42F008020264C1F8104110228F
:101E20008265026C42F0100202640C480C4A0068A1
:101E3000904204D141F8B83F8B60CB60F0BD094AB5
:101E40009042FBD1812041F8B80F8860C860F0BD96
:101E500000C002400080092002000100CC000010F8
:101E6000473F1927473F194710B5FEF7A1FBFEF77B
:101E7000CDFB04494FF40052C1E90020A0F5F42045
:101E8000886010BD0000001006493022C1F8082209
:101E9000C1F81002D1F800028006FBD5D1F8140277
:101EA0007047000000C00820094806210161072191
:101EB000016000214161416202214160C168C9069F
:101EC000FCD400E08168C1684907FBD4002070475A
:101ED0000000034000B50B46024604E0002000F07D
:101EE00005F802F8010B5B1EF8D200BD03498860BB
:101EF000C868C006FCD48868704700000000034032
:101F000000B50B46024603E012F8010BFFF7EEFFA7
:101F10005B1EF9D200BD00002DE9F84F6946384834
:101F200000F056FC8227374C374D384E4FF0220ACE
:101F3000002855D19DF80000800701D400F0B6FDBF
:101F400000BF00BF00BF00BF00BF00BF00BF00BF99
:101F500000BF00BF00BF00BF00BF00BF00BF00BF89
:101F600000BF00BF00BF00BF00BF00BF00BF00BF79
:101F700000BF00BF00BF00BF00BF00BF00BF00BF69
:101F8000DFF88C904FF04008C9F81C806020FFF704
:101F9000ADFFC9F8188000BF00BF00BF00BF00BF81
:101FA00000BF00BF00BF00BF00BF00BF00BF00BF39
:101FB00000BF00BF00BF00BF00BF00BF00BF00BF29
:101FC00000BF00BF00BF00BF00BF00BF00BF00BF19
:101FD00000BF00BF00BF69460E4800F0F9FB38B1F2
:101FE00027607846C5F800A030608220BDE8F88FF1
:101FF000002020602860784630600020F6E700006E
:10200000A0860100800000108400001088000010ED
:102010000080092020A107002DE9F0474FF00009BA
:1020200000BF00BF00BF00BF00BF00BF00BF00BFB8
:1020300000BF00BF00BF00BF00BF00BF00BF00BFA8
:1020400000BF00BF00BF00BF00BF00BF00BF00BF98
:1020500000BF00BF00BF00BF00BF00BF00BF00BF88
:102060004025314EF5619F20FFF740FF0020FFF72C
:102070003DFF00F0FF080020FFF738FFC4B200204A
:10208000FFF734FFC1B2B56100BF00BF00BF00BFA2
:1020900000BF00BF00BF00BF00BF00BF00BF00BF48
:1020A00000BF00BF00BF00BF00BF00BF00BF00BF38
:1020B00000BF00BF00BF00BF00BF00BF00BF00BF28
:1020C00000BF00BF00BF00BF184D194E194FB8F137
:1020D000BF0F03D1252C0AD0262C08D082202860DF
:1020E00021203060784638608220BDE8F0871248B1
:1020F000412912D04FF48002422912D04A2910D02F
:10210000C0F80090002000F0CFFAC5F800907846A3
:10211000C6F8009038600020E7E74FF40011016036
:10212000F0E70260EEE70000008009208000001068
:102130008400001088000010280100102DE9F04FE5
:10214000DFF89480DFF894B089B00F0004464FF0B8
:10215000000628D04FF4805501462A466846FDF710
:10216000E1FFDDE900A105912A46214606A8FDF719
:10217000D9FFDDE906404FF00009BD1BC0F58051D5
:10218000A94200D20D4620B1544517D10599884285
:1021900014D1204600F026F800060FD5D8F800002C
:1021A00009B0BDE8F08F8621C8F800100921CBF8EE
:1021B000001079460A4801608620F1E72E44641C2D
:1021C0004846BE42D9D3C8F800007946CBF8000093
:1021D000034801600020E3E7800000108400001045
:1021E000880000102DE9FC47044601A93A4800F098
:1021F000EFFA3A4D3A4EDFF8EC9048B18220286071
:102200002220794630608220C9F80010BDE8FC87A2
:102210009DF80400800701D400F048FC20208DF8D0
:10222000000020098DF8010020018DF80200002433
:102230008DF8034000BF00BF00BF00BF00BF00BF5C
:1022400000BF00BF00BF00BF00BF00BF00BF00BF96
:1022500000BF00BF00BF00BF00BF00BF00BF00BF86
:1022600000BF00BF00BF00BF00BF00BF00BF00BF76
:1022700000BF00BF4027DFF87080C8F81C70042141
:102280006846FFF73DFEC8F8187000BF00BF00BFEA
:1022900000BF00BF00BF00BF00BF00BF00BF00BF46
:1022A00000BF00BF00BF00BF00BF00BF00BF00BF36
:1022B00000BF00BF00BF00BF00BF00BF00BF00BF26
:1022C00000BF00BF00BF00BF00BF2C607946346074
:1022D0000020C9F8001099E7A086010080000010D6
:1022E0008400001088000010008009204FF4805006
:1022F0007047000001480068704700002801001086
:1023000070B5044600BF00BF00BF00BF00BF00BFE4
:1023100000BF00BF00BF00BF00BF00BF00BF00BFC5
:1023200000BF00BF00BF00BF00BF00BF00BF00BFB5
:1023300000BF00BF00BF00BF00BF00BF00BF00BFA5
:1023400000BF00BF4025174EF5610520FFF7CEFD09
:102350000020FFF7CBFD2070B56100BF00BF00BFBC
:1023600000BF00BF00BF00BF00BF00BF00BF00BF75
:1023700000BF00BF00BF00BF00BF00BF00BF00BF65
:1023800000BF00BF00BF00BF00BF00BF00BF00BF55
:1023900000BF00BF00BF00BF00BF207800F00100F9
:1023A00070BD00000080092070B5044600BF00BF6A
:1023B00000BF00BF00BF00BF00BF00BF00BF00BF25
:1023C00000BF00BF00BF00BF00BF00BF00BF00BF15
:1023D00000BF00BF00BF00BF00BF00BF00BF00BF05
:1023E00000BF00BF00BF00BF00BF00BF4025174EA9
:1023F000F5610520FFF77AFD0020FFF777FD2070DB
:10240000B56100BF00BF00BF00BF00BF00BF00BF7D
:1024100000BF00BF00BF00BF00BF00BF00BF00BFC4
:1024200000BF00BF00BF00BF00BF00BF00BF00BFB4
:1024300000BF00BF00BF00BF00BF00BF00BF00BFA4
:1024400000BF207800F0010070BD0000008009206E
:1024500070B50C4D0C4E0D4C2AB100F019F8000669
:1024600009D5206870BD8620206009202860784644
:102470003060862070BD0020206028607846306083
:10248000002070BD84000010880000108000001043
:102490002DE9FC5F3D4D3E4E3E4F5FEA020A8B4602
:1024A00004464FF000080DD001A93B4800F090F918
:1024B00080B18220286021203060784638608220F8
:1024C000BDE8FC9FC5F800807846C6F800803860FB
:1024D0000020F5E703208DF80000200C8DF80100A6
:1024E000200A8DF802008DF8034000BF00BF00BF36
:1024F00000BF00BF00BF00BF00BF00BF00BF00BFE4
:1025000000BF00BF00BF00BF00BF00BF00BF00BFD3
:1025100000BF00BF00BF00BF00BF00BF00BF00BFC3
:1025200000BF00BF00BF00BF00BF1C4C4FF0400900
:10253000C4F81C9004216846FFF7E2FC5146584657
:10254000FFF7C8FCC4F8189000BF00BF00BF00BF71
:1025500000BF00BF00BF00BF00BF00BF00BF00BF83
:1025600000BF00BF00BF00BF00BF00BF00BF00BF73
:1025700000BF00BF00BF00BF00BF00BF00BF00BF63
:1025800000BF00BF00BF00BF9CE70000800000103C
:102590008400001088000010A0860100008009203F
:1025A0002DE9FC478A46044601A93A4800F010F993
:1025B000394D3A4EDFF8E89048B182202860222059
:1025C000794630608220C9F80010BDE8FC870320FE
:1025D0008DF8000020098DF8010020018DF802001F
:1025E00000248DF8034000BF00BF00BF00BF00BF44
:1025F00000BF00BF00BF00BF00BF00BF00BF00BFE3
:1026000000BF00BF00BF00BF00BF00BF00BF00BFD2
:1026100000BF00BF00BF00BF00BF00BF00BF00BFC2
:1026200000BF00BF00BF4027DFF87880C8F81C70EB
:1026300004216846FFF764FCB9015046FFF74AFCE5
:10264000C8F8187000BF00BF00BF00BF00BF00BFC8
:1026500000BF00BF00BF00BF00BF00BF00BF00BF82
:1026600000BF00BF00BF00BF00BF00BF00BF00BF72
:1026700000BF00BF00BF00BF00BF00BF00BF00BF62
:1026800000BF00BF2C60794634600020C9F80010FC
:102690009BE70000A086010080000010840000106D
:1026A000880000100080092070B5064600BF00BFFA
:1026B00000BF00BF00BF00BF00BF00BF00BF00BF22
:1026C00000BF00BF00BF00BF00BF00BF00BF00BF12
:1026D00000BF00BF00BF00BF00BF00BF00BF00BF02
:1026E00000BF00BF00BF00BF00BF00BF4024374D88
:1026F000EC615020FFF7FAFBAC6100BF00BF00BFE8
:1027000000BF00BF00BF00BF00BF00BF00BF00BFD1
:1027100000BF00BF00BF00BF00BF00BF00BF00BFC1
:1027200000BF00BF00BF00BF00BF00BF00BF00BFB1
:1027300000BF00BF00BF00BF00BF00BF00BF00BFA1
:1027400000BF00BF00BF00BF00BF00BF00BF00BF91
:1027500000BF00BF00BF00BF00BF00BF00BF00BF81
:1027600000BF00BF00BF00BF00BF00BF00BF00BF71
:1027700000BF00BF00BF00BF00BFEC610120FFF73A
:10278000B5FBB000FFF7B2FBAC6100BF00BF00BFFC
:1027900000BF00BF00BF00BF00BF00BF00BF00BF41
:1027A00000BF00BF00BF00BF00BF00BF00BF00BF31
:1027B00000BF00BF00BF00BF00BF00BF00BF00BF21
:1027C00000BF00BF00BF00BF00BF70BD0080092078
:1027D0002DE9F041084C0F460646A56806E0A068C2
:1027E000401BB04202D30120BDE8F0813846FFF71C
:1027F00087FD0028F3D1F7E7000009402DE9F041FB
:10280000084C0F460646A56806E0A068401BB0428B
:1028100002D30120BDE8F0813846FFF7C5FD00284E
:10282000F3D1F7E7000009402DE9F04F89B0DFF858
:10283000D080DFF8D0B05FEA02094FF000060791C0
:102840000FD04FF4805501462A466846FDF76AFCD2
:10285000DDE90047284602F0BDF85FEA000A0DD026
:1028600017E08621C8F800100921CBF8001079463E
:1028700025480160862009B0BDE8F08F8221C8F8A4
:1028800000102221CBF8001079461F4801608220F9
:10289000F1E7A9EB0605C7F58050A84200D205462E
:1028A000B5F5805F04D020465146FFF779FE80B928
:1028B0002046FFF797FC60B907982A46811907EB75
:1028C0000A00FDF739FC2E442046514600F044FA38
:1028D00028B1504601F0CEFFD8F80000CBE7002722
:1028E000641C4E45D5D3504601F0C4FF0020C8F803
:1028F00000007946CBF80000034801600020BAE7E9
:102900008000001084000010880000102DE9FE43B4
:102910000F46044602A93A48FFF75AFF394D3A4E8E
:10292000DFF8E88048B182202860222079463060B4
:102930008220C8F80010BDE8FE839DF808008007DB
:1029400001D400F0B3F802208DF80000200C8DF8BF
:102950000100200A8DF802008DF803408DF8047004
:1029600000BF00BF00BF00BF00BF00BF00BF00BF6F
:1029700000BF00BF00BF00BF00BF00BF00BF00BF5F
:1029800000BF00BF00BF00BF00BF00BF00BF00BF4F
:1029900000BF00BF00BF00BF00BF00BF00BF00BF3F
:1029A00040241B4FFC6105216846FFF7A9FABC6172
:1029B00000BF00BF00BF00BF00BF00BF00BF00BF1F
:1029C00000BF00BF00BF00BF00BF00BF00BF00BF0F
:1029D00000BF00BF00BF00BF00BF00BF00BF00BFFF
:1029E00000BF00BF00BF00BF00BF00BF00BF00BFEF
:1029F0000020286079463060C8F800109BE700008E
:102A0000A0860100800000108400001088000010E3
:102A10000080092070B500BF00BF00BF00BF00BF2D
:102A200000BF00BF00BF00BF00BF00BF00BF00BFAE
:102A300000BF00BF00BF00BF00BF00BF00BF00BF9E
:102A400000BF00BF00BF00BF00BF00BF00BF00BF8E
:102A500000BF00BF00BF4025134CE5610420FFF715
:102A600045FAA56100BF00BF00BF00BF00BF00BFA7
:102A700000BF00BF00BF00BF00BF00BF00BF00BF5E
:102A800000BF00BF00BF00BF00BF00BF00BF00BF4E
:102A900000BF00BF00BF00BF00BF00BF00BF00BF3E
:102AA00000BF00BF70BD00000080092070B500BFEE
:102AB00000BF00BF00BF00BF00BF00BF00BF00BF1E
:102AC00000BF00BF00BF00BF00BF00BF00BF00BF0E
:102AD00000BF00BF00BF00BF00BF00BF00BF00BFFE
:102AE00000BF00BF00BF00BF00BF00BF00BF402548
:102AF000134CE5610620FFF7F9F9A56100BF00BF9F
:102B000000BF00BF00BF00BF00BF00BF00BF00BFCD
:102B100000BF00BF00BF00BF00BF00BF00BF00BFBD
:102B200000BF00BF00BF00BF00BF00BF00BF00BFAD
:102B300000BF00BF00BF00BF00BF00BF70BD0000EE
:102B4000008009202DE9F05F114EDFF84890DFF892
:102B500048A0150083460F464FF000080ED0002411
:102B60000AE0395D0BEB0400FFF7D0FE000602D54A
:102B70003068BDE8F09F641CAC42F2D3C6F8008018
:102B80007946C9F800800020CAF80010F1E700007B
:102B90008000001084000010880000102DE9FF4F15
:102BA0008DB00D46DDF868900026684C07935FEA0B
:102BB00009013ED04FF4805701463A466846FDF77A
:102BC000B1FADDE900B10C913A46691C6846FDF79F
:102BD000A9FADDE90010CDE904013A4668460F99EB
:102BE000FDF7A0FADDE90085A9EB0607C5F58050E1
:102BF000B84200D2074625B1D8457DD10C98854210
:102C00007AD14FF4805001F0E5FE5FEA000A1CD053
:102C1000D84550D10C9885424DD12A464FEA08300C
:102C20005146FFF735FC000619D5504601F022FE4B
:102C30007AE08620206046480921016078464549AF
:102C40000860862011B0BDE8F08F822020604048E7
:102C50002221016079463F4801608220F2E7059811
:102C6000804509D1049901EB0030C1F580525144EF
:102C7000FFF70EFC0006D8D44046FFF7B3FA000673
:102C8000D3D407983A46811905EB0A00FDF754FAA8
:102C9000EA194FEA08305146FFF754FF0006C4D442
:102CA0000599884533D1049800EB01300499C1F5AA
:102CB0008052514427E0059988450AD1049800EBD9
:102CC00001300499C1F580525146FFF7E1FB00063F
:102CD000ABD44046FFF786FA0006A6D407983A46DA
:102CE00081190F983044FFF72DFF00069DD40599F8
:102CF00088450CD1049800E00DE000EB0130049908
:102D0000C1F580525146FFF71DFF00068DD4504695
:102D100001F0B0FD0AE007983A4681190F98304457
:102D2000FFF710FF000601D520688BE73E44002521
:102D300008F101084E45FFF457AF05490020206017
:102D4000086078460349086000207BE78000001097
:102D500084000010880000102DE9F34F83B0044672
:102D600001A97148FFF734FD704D714E714F4FF05E
:102D7000820818B12120C5F800806CE09DF804009D
:102D8000800701D4FFF792FEAD208DF800002009E6
:102D90008DF8010020018DF802004FF0000B8DF836
:102DA00003B000BF00BF00BF00BF00BF00BF00BF37
:102DB00000BF00BF00BF00BF00BF00BF00BF00BF1B
:102DC00000BF00BF00BF00BF00BF00BF00BF00BF0B
:102DD00000BF00BF00BF00BF00BF00BF00BF00BFFB
:102DE00000BFDFF854914FF0400A5446C9F81CA0C8
:102DF00004216846FFF784F802210498FFF780F861
:102E0000C9F8184000BF00BF00BF00BF00BF00BF2F
:102E100000BF00BF00BF00BF00BF00BF00BF00BFBA
:102E200000BF00BF00BF00BF00BF00BF00BF00BFAA
:102E300000BF00BF00BF00BF00BF00BF00BF00BF9A
:102E400000BF00BF022401A93748FFF7C1FC48B109
:102E50002220C5F80080306078463860822005B0B6
:102E6000BDE8F08F00BF00BF00BF00BF00BF00BFC4
:102E700000BF00BF00BF00BF00BF00BF00BF00BF5A
:102E800000BF00BF00BF00BF00BF00BF00BF00BF4A
:102E900000BF00BF00BF00BF00BF00BF00BF00BF3A
:102EA00000BF00BFC9F81CA0AD20FFF71FF80498B1
:102EB00002212044FFF724F8C9F818A000BF00BF82
:102EC00000BF00BF00BF00BF00BF00BF00BF00BF0A
:102ED00000BF00BF00BF00BF00BF00BF00BF00BFFA
:102EE00000BF00BF00BF00BF00BF00BF00BF00BFEA
:102EF00000BF00BF00BF00BF00BF00BFA41CA4B242
:102F0000B4F5805F9FD301A90748FFF761FC002853
:102F10007FF430AFFFF77EFDC5F800B07846C6F805
:102F200000B0386000209AE7A08601008000001001
:102F30008400001088000010008009204FF48050A9
:102F400070474FF4800070472DE9F04F89B0DFF8EB
:102F5000D080DFF8D0B05FEA02094FF00006079199
:102F60000FD04FF4805501462A466846FDF7DAF83F
:102F7000DDE90047284601F02DFD5FEA000A0DD08B
:102F800017E08621C8F800100921CBF80010794617
:102F900025480160862009B0BDE8F08F8221C8F87D
:102FA00000102221CBF8001079461F4801608220D2
:102FB000F1E7A9EB0605C7F58050A84200D2054607
:102FC000B5F5805F04D020465146FFF7E9FA80B995
:102FD0002046FFF707F960B907982A46811907EBE1
:102FE0000A00FDF7A9F82E442046514600F094FA55
:102FF00028B1504601F03EFCD8F80000CBE700278E
:10300000641C4E45D5D3504601F034FC0020C8F86E
:1030100000007946CBF80000034801600020BAE7C1
:103020008000001084000010880000102DE9FF4788
:1030300003A93A48FFF7E2FB394D3A4EDFF8E89032
:1030400050B1822028602120794630608220C9F862
:10305000001004B0BDE8F0879DF80C00800701D493
:10306000FFF724FD42208DF800000024CDF8014038
:10307000CDF80540ADF8094000BF00BF00BF00BF5C
:1030800000BF00BF00BF00BF00BF00BF00BF00BF48
:1030900000BF00BF00BF00BF00BF00BF00BF00BF38
:1030A00000BF00BF00BF00BF00BF00BF00BF00BF28
:1030B00000BF00BF00BF00BF4027DFF87080C8F826
:1030C0001C700B216846FEF71BFFC8F8187000BF84
:1030D00000BF00BF00BF00BF00BF00BF00BF00BFF8
:1030E00000BF00BF00BF00BF00BF00BF00BF00BFE8
:1030F00000BF00BF00BF00BF00BF00BF00BF00BFD8
:1031000000BF00BF00BF00BF00BF00BF00BF2C60FA
:10311000794634600020C9F800109AE7A0860100C3
:10312000800000108400001088000010008009203A
:103130002DE9F34F85B0044603A96D48FFF75EFB08
:103140006C4D6D4E6D4F4FF0820B18B12120C5F8BC
:1031500000B060E0FFF7AAFC42208DF800004FF0BD
:10316000000ACDF801A0CDF805A0ADF809A000BF78
:1031700000BF00BF00BF00BF00BF00BF00BF00BF57
:1031800000BF00BF00BF00BF00BF00BF00BF00BF47
:1031900000BF00BF00BF00BF00BF00BF00BF00BF37
:1031A00000BF00BF00BF00BF00BF00BF00BFDFF80F
:1031B00050914FF04008C9F81C800B216846FEF77B
:1031C0009FFEC9F8188000BF00BF00BF00BF00BF4E
:1031D00000BF00BF00BF00BF00BF00BF00BF00BFF7
:1031E00000BF00BF00BF00BF00BF00BF00BF00BFE7
:1031F00000BF00BF00BF00BF00BF00BF00BF00BFD7
:1032000000BF00BF00BF03A93948FFF7F7FA48B174
:103210002220C5F800B0306078463860822007B0C0
:10322000BDE8F08F9DF80C00800701D4FFF73EFC4D
:1032300002208DF80000200C8DF80100200A8DF886
:10324000020006988DF803408DF8040000BF00BF0F
:1032500000BF00BF00BF00BF00BF00BF00BF00BF76
:1032600000BF00BF00BF00BF00BF00BF00BF00BF66
:1032700000BF00BF00BF00BF00BF00BF00BF00BF56
:1032800000BF00BF00BF00BF00BF00BF4446C8462C
:10329000C9F81C4005216846FEF732FEC8F8184000
:1032A00000BF00BF00BF00BF00BF00BF00BF00BF26
:1032B00000BF00BF00BF00BF00BF00BF00BF00BF16
:1032C00000BF00BF00BF00BF00BF00BF00BF00BF06
:1032D00000BF00BF00BF00BF00BF00BF00BF00BFF6
:1032E000C5F800A07846C6F800A03860002096E730
:1032F000A0860100800000108400001088000010EB
:10330000008009202DE9F05F114EDFF84890DFF8CA
:1033100048A0150083460F464FF000080ED0002449
:103320000AE0395D0BEB0400FFF702FF000602D54F
:103330003068BDE8F09F641CAC42F2D3C6F8008050
:103340007946C9F800800020CAF80010F1E70000B3
:103350008000001084000010880000102DE9FF4F4D
:103360008DB00D46DDF868900026684C07935FEA43
:1033700009013ED04FF4805701463A466846FCF7B3
:10338000D1FEDDE900B10C913A46691C6846FCF7B4
:10339000C9FEDDE90010CDE904013A4668460F99FF
:1033A000FCF7C0FEDDE90085A9EB0607C5F58050F6
:1033B000B84200D2074625B1D8457DD10C98854248
:1033C0007AD14FF4805001F005FB5FEA000A1CD06F
:1033D000D84550D10C9885424DD12A464FEA083045
:1033E0005146FFF755F8000619D5504601F042FA4C
:1033F0007AE08620206046480921016078464549E8
:103400000860862011B0BDE8F08F8220206040481F
:103410002221016079463F4801608220F2E7059849
:10342000804509D1049901EB0030C1F58052514427
:10343000FFF72EF80006D8D44046FEF7D3FE00066C
:10344000D3D407983A46811905EB0A00FCF774FEBD
:10345000EA194FEA08305146FFF754FF0006C4D47A
:103460000599884533D1049800EB01300499C1F5E2
:103470008052514427E0059988450AD1049800EB11
:1034800001300499C1F580525146FFF701F800065A
:10349000ABD44046FEF7A6FE0006A6D407983A46EF
:1034A00081190F983044FFF72DFF00069DD4059930
:1034B00088450CD1049800E00DE000EB0130049940
:1034C000C1F580525146FFF71DFF00068DD45046CE
:1034D00001F0D0F90AE007983A4681190F98304474
:1034E000FFF710FF000601D520688BE73E4400255A
:1034F00008F101084E45FFF457AF05490020206050
:10350000086078460349086000207BE780000010CF
:1035100084000010880000102DE9F34F0024494D6D
:10352000494E4A4FC3B080464FF0820A4FF0210BFC
:10353000A14641A94648FFF761F900286ED19DF8E0
:103540000401800701D4FFF7B1FA02208DF80000D2
:103550004FEA18108DF8010004EB08108DF80200F6
:1035600044988DF8039000EB04214FF4807201A879
:10357000FCF7E2FD00BF00BF00BF00BF00BF00BFFF
:1035800000BF00BF00BF00BF00BF00BF00BF00BF43
:1035900000BF00BF00BF00BF00BF00BF00BF00BF33
:1035A00000BF00BF00BF00BF00BF00BF00BF00BF23
:1035B00000BF00BF40202749C8614FF482716846B0
:1035C000FEF79EFC23494020886100BF00BF00BF7A
:1035D00000BF00BF00BF00BF00BF00BF00BF00BFF3
:1035E00000BF00BF00BF00BF00BF00BF00BF00BFE3
:1035F00000BF00BF00BF00BF00BF00BF00BF00BFD3
:1036000000BF00BF00BF00BF00BF641CE4B2102CAD
:103610008FD341A90E48FFF7F1F848B1C5F800A0D3
:103620007846C6F800B03860822045B0BDE8F08F1B
:10363000FFF7F0F9C5F800907846C6F800903860BA
:103640000020F2E7800000108400001088000010C5
:10365000A086010000800920F8B51446074E0A46EE
:103660000B19716800258B4200D90A1B0346009490
:103670003068FDF713F92846F8BD0000000000107F
:1036800070B5034608468D180549002449688D42E7
:1036900000D9881A1946FDF7CBF8204670BD000006
:1036A0000000001002480168491C016070470000DA
:1036B000EC00001010B54FF0E024054860611F21B8
:1036C0006017FEF747FA0020A0610720206110BDB7
:1036D000BFD40100094810B50221416000210167F3
:1036E00041611D22C260C16301214160FFF7E2FF19
:1036F0000221C81EFEF72EFA002010BD000009406E
:10370000F0B54C48D0F804114FF00002CB054A49FF
:1037100028D4D0F80C31DC07484B03D0D0F8A041B6
:10372000640660D5D0F80441E40605D0D0F8044121
:1037300004F01F04B3FBF4F40C60D0F8A851ED06BC
:103740000ED0D0F8A85105F01F05B3FBF5F34B6080
:10375000D0F8003103F001035B1CB4FBF3F331E05C
:103760000023F4E7D0F88830DB053CD5D0F80C31E5
:10377000DB0703D0D0F8A0315B0634D5D0F8883011
:10378000D0F8044103F01F0314F01F05D0F8A8413E
:10379000D0F8006104F01F0406F0010603F10103F4
:1037A00006F1010603D0254F5F43B7FBF5F50D6029
:1037B00024B1224F7B43B3FBF4F300E000234B60C2
:1037C000B5FBF6F3C1F80830D0F80831DB05D0F8C6
:1037D00008311CD513F01F0303D0042B07D0062B90
:1037E00005D0CA60F0BD0A604A608A60ECE7D0F894
:1037F0008820D0F8083102F01F02D0F80C0103F045
:103800001F030E48521C4243B2FBF3F00FE09B052E
:10381000E7D5D0F80C21D20702D0D0F8A80001E0FB
:10382000D0F88800054A00F01F00401C5043C860D3
:10383000F0BD000000C00F40DC000010001BB7000E
:10384000264810B42021C0F8A01100BFD0F8A01164
:103850004906FBD50121C0F80C110922C0F88420CB
:10386000C0F88010AA22C0F88C205523C0F88C30F4
:10387000D0F888406405FBD52324C0F8A440C0F8E4
:10388000A010C0F8AC20C0F8AC3000BFD0F8A82021
:103890005205FBD540F20112C0F8042140F201228A
:1038A000C0F80821C0F800110221C0F8B4110421A9
:1038B000C0F8A8110A49C0F8C4100021C0F8C81106
:1038C000D0F8B02142F00302C0F8B02145F23A022C
:1038D00002600448016010BCFFF712BF00C00F4037
:1038E000FE9FF8F708ED00E010B54FF040210120F1
:1038F0000860FCF79FFC10BD00B5FCF7F3FC044921
:103900005DF804EB41EA0040891300F019BD0000A6
:103910000005400010B502468078FCF7E3FC0B4937
:10392000D1F84432012484402343C1F84432C1F821
:1039300048029088C1F84C02D1F80002C005FBD5BE
:103940004FF48070C1F8080210BD000000C00820CC
:1039500010B500B101204FF4807444EA00410748DB
:1039600000F0EEFC06480321C0F84412D0F8001223
:10397000C905FBD5C0F8084210BD00000005D800FD
:1039800000C0082010B5040001D0012000E0002094
:103990004FF4807141EA0041054800F0D1FC05492F
:1039A0004FF480200CB1886310BDC86310BD0000C7
:1039B0000005FE000080092010B5084CA288402AAE
:1039C00000D940228020216800F062FC2168014477
:1039D0002160A188081AA08010BD00000C01001011
:1039E00010B5064C0020216800F02CFA2168014433
:1039F0002160A188081AA08010BD00000C010010F1
:103A000000B5FCF76FFC04495DF804EB41EA0040A7
:103A1000024900F095BC00000005400000012000B4
:103A200000B5FCF75FFC04495DF804EB41EA004097
:103A3000891300F085BC0000000540002DE9F0412D
:103A40004A4C0027A4F108062178A4F11C05082897
:103A500064D2DFE800F0630465746363868400F079
:103A6000F7FB2078C009FCF7CCFCE088B080207818
:103A7000C0F34111F1BB61780C294BD2DFE801F0B2
:103A800006094A0B4A101B1E2026324300F0B6F8E6
:103A90004EE0002000E0012000F062FA50B306E0A2
:103AA00010F01F0F36D1A07840F080002870BDE8DC
:103AB000F04100F0D3BB00F065F839E000202AE0C7
:103AC00010F01F0F26D129481B381AE010F01F0FE5
:103AD00020D100F08DFA68B100F0C0FBBDE8F041E4
:103AE000FCF78EBC00F01F00012813D1687808B1E4
:103AF000207900E00EE0A97888420BD21B490C39EE
:103B0000084430601DE000F01F00012802D100F0E1
:103B100017FBC3E7802000F08BFBB780BDE8F08186
:103B2000080608D4B0880028F8D0FFF759FFB088FD
:103B30000028EFD0F2E7BDE8F04100F095BB0806A1
:103B400003D5BDE8F041FFF737BF28780106E5D57A
:103B500000F07F002870BDE8F04100F0EDB9802052
:103B600000E00020BDE8F041FFF7C6BE14010010E0
:103B7000022803D0032803D1FDF736B8FDF756B865
:103B800070470000194810B5007810F01F0F174853
:103B9000C07829D115490839012806D0134A0228CE
:103BA000937806D003281FD112E011480860122034
:103BB00012E01048002204E004780CB1448820444C
:103BC000521C9342F8D1027872B10860408803E039
:103BD00009481844086000788A88824200D98880A1
:103BE000FFF7EAFE012010BD002010BD14010010F7
:103BF000585200006A5200008B52000070B51D48F8
:103C00001C4D0078A5F1080510F01F040AD01948D2
:103C1000A5F11401184B4A780079012C06D0022C2A
:103C200026D109E01348183828601DE002B38978CE
:103C300088421DD2002015E000F08F04200605D533
:103C400004F00F064FF48030B04001E00120A040A6
:103C50000AB922070CD18A68024209D0C968014218
:103C6000E8D0012018802B60FFF7A6FE012070BD70
:103C7000002070BD14010010341D00102DE9F0412A
:103C80002F4DD5F80032C5F80832180721D52D4838
:103C900000F048FB2C48FEF7F7F8C10605D500F008
:103CA00007F9BDE8F04100F03BB9810705D5BDE853
:103CB000F04100F0010000F07FB8010709D540078E
:103CC00003D5BDE8F04100F0D5BABDE8F04100F001
:103CD00031B91E4E58074FF001071DD4BDE8F081E1
:103CE0005FF00004D5F8302207FA04F10A4210D040
:103CF0006008C5F8381200BFD5F800128906FBD558
:103D0000D5F81412E2070CD056F8201009B10320A0
:103D10008847641C202CE5D3D5F830020028DFD179
:103D2000DCE73CB9490705D5316819B1012088475E
:103D30000124D7E756F820100029EAD00220E7E74F
:103D400000C008200005FE000002FE00FC5200003A
:103D500030B5154C1A202060221D116830EA01018F
:103D6000FBD1124901234B678B67114D0023C5F826
:103D700010318A23C1F8F8302060116830EA01015F
:103D8000FBD14FF0E0214FF08070C1F88002094B69
:103D9000202283F80024C1F8000100F089F8BDE872
:103DA0003040002000F0C8B8F4CF082000C0024026
:103DB00000C0082018E000E0002802D101490120DD
:103DC000487070471C01001070B5194C607820B322
:103DD0000026184D012810D002280DD1A86861686E
:103DE000401A1549884215D31448406B400011D53C
:103DF0000120FFF7C7FD667070BDA8686168401AB2
:103E00000F498842F8D30020FFF7BCFDA868606026
:103E10000220607026700C2005E020780028EBD18D
:103E2000012020700D20BDE87040FCF7FDBD0000B2
:103E30001C01001000000940A0860100008009203C
:103E400040420F0000F00F02012370B503EB820324
:103E5000154AC2F8283200BFD2F820321C05FBD523
:103E6000C3F309030024DD1C05E000BFD2F818628B
:103E700041F8046B641CB4EB950FF7D30021C2F832
:103E8000281241F24821C140C9070AD1FCF72AFA99
:103E90004FF4A06141EA004000F044FA034800F00A
:103EA00041FA184670BD000000C008200005F2006D
:103EB0000D480021C0F848124021C0F84C120122E0
:103EC000C0F84822C0F84C12D0F80012C905FBD542
:103ED0004FF0FF31C0F83812C0F83412C0F80812A1
:103EE0000C21C0F80412704700C0082004480021CB
:103EF0004FF00112818001704170C0E902217047CA
:103F0000F800001000B5FCF7EDF904495DF804EB8A
:103F100041EA0040891300F013BA00000005400098
:103F200010B5FFF7E3FF02490020487010BD000004
:103F30001C0100107047000030B50749074D41EAE9
:103F400000442146284600F0FBF921462846BDE8FA
:103F5000304000F0F5B90000000180000005D000FD
:103F600070B502462148A0F11C04017811F01F032E
:103F70000146498804D0012B29D0022B27D111E01A
:103F8000012924D132B1012000F080F9A08840F04D
:103F9000020005E0002000F079F9A08820F002007E
:103FA000A08021E0007900F08F00030605D500F025
:103FB0000F034FF480359D4001E001258540637873
:103FC0002BB1030703D0A3682B4200D009B1002016
:103FD00070BD22B100F02CF9E068284303E0FFF740
:103FE0008BFCE068A843E060012070BD1401001064
:103FF0002DE9F84F504F00200090B8784FF000099D
:104000004FF0010A4FF4803BA7F11C0600286AD04C
:104010004A4C64E06078022804D0042840D0052887
:104020005BD140E06179B878814237D170702079F6
:10403000B070414900200C3901F80090401C042860
:10404000FAD301254FEA06080AFA05F0D8F8081055
:10405000084202D02846FFF7D3FCD8F808100BFA24
:1040600005F0084203D045F08000FFF7C9FC6D1C45
:10407000102DE9D34FF00110C8E902090120FFF724
:1040800067FCE0794006B8F8040002D540F0010072
:1040900001E020F00100A8F804001EE060881DE0A7
:1040A000E078009019E00098B8B9A07800F08F058A
:1040B000280604D505F00F010BFA01F001E00AFA19
:1040C00005F0B16801432046B160FFF723FC2846A4
:1040D000FFF7A6FC2846FFF715FF20780444207858
:1040E000002897D11FE086F8019001245546D84654
:1040F000B16805FA04F0084202D02046FFF780FCC0
:10410000B16808FA04F0084203D044F08000FFF7D9
:1041100077FC641C102CEBD34FF00110C6E90209A8
:104120000020FFF715FCB8787178884202D1012091
:10413000BDE8F88F0020FBE7140100106A52000070
:104140002DE9FC5F384D00273E466878BB46B846EF
:10415000002866D0BA46354C05F11C095DE0607850
:10416000022804D0042808D0052854D119E0607929
:10417000697888424FD060884EE0A77899F804109B
:10418000E6784FF00008B94245D199F80200B042F4
:1041900041D125484FF0010A103010F807B0C6553C
:1041A00039E099F80410B94235D1A17801F08F01B6
:1041B0000191090605D5019901F00F024FF48031F4
:1041C00001E0019A01219140009199F80200B0426A
:1041D00013D1A8680843A860E96800988143204685
:1041E000E960FFF797FB0198FFF71AFC0198FFF7CA
:1041F00089FE009948EA01080DE05E450BD118EAF6
:10420000010F08D1A8688843A860E8688843E8607F
:104210000198FFF7F5FB20780444207800289ED110
:104220005046BDE8FC9F0000F80000106A520000F4
:1042300000B5FCF757F804495DF804EB41EA00408B
:10424000024900F07DB800000005400000010100B7
:1042500001490020FFF7F6BD1401001000221146AD
:10426000802000F015B8000001490020FFF7EABDEA
:10427000341D0010034801214170034989684160E1
:10428000704700001C01001000000940704700004A
:1042900070B513460546134C00F00F00022202EBE6
:1042A0008000C4F82802C4F824320020DA1C04E09C
:1042B00051F8046BC4F81C62401CB0EB920FF7D3AA
:1042C0000020C4F828022846FCF70CF84FF4A0613F
:1042D00041EA004000F026F8034800F023F81846B1
:1042E00070BD000000C008200005FA00EFF3108048
:1042F00010F0010F72B64FF080404FF000020270D4
:104300004FF0AA0202724FF0550303724FF0FF0400
:1043100044604FF0030404700272037200D162B66D
:10432000FEE7000005491022C1F80822C1F810027A
:10433000D1F80002C006FBD57047000000C008207D
:10434000094A1023C2F80832C2F81002D2F800025B
:10435000C006FBD5C2F80832C2F81012D2F800022B
:10436000C006FBD57047000000C0082002E008C866
:10437000121F08C1002AFAD170477047002001E0DF
:1043800001C1121F002AFBD1704700000B4910B574
:10439000486980040CD40A4A906843F698239468CC
:1043A000241A9C42FBD34869800401D4012010BD2B
:1043B0000520FCF739FB002010BD0000008009201B
:1043C00000000940F0B505460020034602462B4C8C
:1043D0004FF4007700E05B1CEE5C46B102EB030C8F
:1043E000A4440CF5805C9CF800C8B445F3D0032BC2
:1043F0003FD302F5C0502044037F457FC67F03EBC7
:104400000523857F2D0405EB06652B4451EA030542
:104410002BD021B91A49496840318B4225D8194B14
:1044200000215518254405F5805595F800585D5430
:10443000491C0C29F5D3817EC27E01EB0221027D4D
:10444000407D120402EB00600C18204600F0F8FAE0
:1044500040F6F57502E000BF00F0F2FAC11EA94275
:10446000FAD3A0F57061FF3901D00020F0BD2046DD
:10447000F0BD2032BA42AFD3F0BD00009101001070
:104480008C000010FD1B001070B50D4CA6680420B8
:10449000FCF7CAFA0B4D02E0FFF778FF48B1A068BD
:1044A000801BA842F8D308E0FFF770FF08B1012095
:1044B00070BDA068801BA842F6D3002070BD00002C
:1044C0000000094080841E008AB046208DF8140048
:1044D0004FF000098DF8179036208DF81500B24A7C
:1044E00034208DF816001068CA464FF6FF031840B6
:1044F000AE4B40F4807018431060AD48AE49B14DEA
:10450000C0F80090AB480068A0F56C50FF38086018
:10451000AA4900F5E0500860A949400A0860F8205F
:104520002870FF206870A870FBF7A2FEA74CA64A6F
:10453000002094F9051052F821102A1802F5805233
:104540000B5C401C82F800386028F6D34FF4E1750C
:10455000294640F24910FBF7A1FE294640F29F1080
:10456000FBF79CFE4FF4005BDFF864825D46207829
:1045700008B1FFF729FCA07928B1012819D02078CB
:1045800000286ED000E10A20FCF74EFAFBF73CFF52
:1045900018B100BFFCF7F2F9E9E70120A0715D4610
:1045A00084F803A00620FCF73FFA0A20FCF73CFA47
:1045B000DDE7192229468648FCF70DFB98F818001C
:1045C00000287CD098F80000062873D2DFE800F0BD
:1045D00072030B46464A40F2044000880390D8F824
:1045E0000410814266D098F809104FF00109404646
:1045F00001295FD1D0F80A1019B976498969C0F844
:104600000A100026804617E00720FCF70DFAD7F8BD
:104610000E00B846871B402F00D94027A9193A46FB
:104620006D481931FCF7D7FAD8F80A003A463044F9
:10463000694900F049FB3E44D8F80E004746B042B5
:10464000E2D83978012935D14FF0E0220906C2F8C5
:104650008011D7F80A0000F0DFF82BE04FF00109D5
:104660002BE08AE098F809104FF00109032924D1C2
:1046700050495A4A00260B68136016E00720FCF7E1
:10468000D3F9D7F80E00871B402F00D94027A9196E
:104690003A4651481931FCF79EFA46483A460068B6
:1046A00081194D48FEF7D8FF3E44D8F80E00474622
:1046B000B042E3D898F8180008B1464600E01CE084
:1046C00098F80800C00613D54449012203A8C1F890
:1046D00000B005F11801CDF80CA0FEF7D1FF30783D
:1046E00020B1C8214FF47A70FBF7D8FD307E20B19D
:1046F000307A800701D5FFF7F9FDD8F80E001B3599
:1047000005443348FCF76AF948B302203449A071E4
:104710005D4681F800A00B20FCF786F9B9F1000F87
:104720001DD030484FF00009816842F21072836852
:104730005B1A9342FBD34FF42F714FF47A70FBF75F
:10474000ADFD29494869400305D5486D400502D5AE
:104750000020099001E0099808B9FFF7C7FDE0784B
:10476000401CC0B2E0700C2802D30120A07011E7F9
:10477000A07800283FF410AF0CE701202070FFF76D
:10478000E7FA0120FFF7FEF8154800780028F1D07D
:10479000002105A8FFF716FE0028EBD084F806A03C
:1047A0005D4684F803A0E2E60CED00E00000FA05A7
:1047B000C000001008000010B0000010A800001099
:1047C000AC00001091010010740000100C000010EB
:1047D000780100106851000038010010000000103E
:1047E0007C0000100000094000800920084A3423A2
:1047F0001360C2E9010107484FF47A710068B0FB09
:10480000F1F0D06002F11401104600F05BB8000036
:104810000C1C0010DC00001072B60349034A014072
:104820001160FBF769BC000080FFFF1F08ED00E08E
:1048300010B572B606240E4951F82420824212D9CE
:104840000B49783951F82410814207D12146084696
:1048500000F01EF921460846FFF7C8FF214608462A
:1048600000F016F902E0641C1D2CE5D962B610BDFB
:10487000E051000010B5002821D0114B0022001F8C
:10488000196803E0814203D80A4649680029F9D132
:1048900052B11368841A9C4204D100681844106015
:1048A000104602E0506000E0186039B102680B1A4F
:1048B000934203D10B681A4402604968416010BDFD
:1048C0003001001030B4074C054A0323C4F8B0315E
:1048D000136843F480331360034A30BC1047000070
:1048E00088C10F4000C00F40F11FFF1F334C00264E
:1048F000FF202660A680A6716071FEF7A1FFFDF77C
:1049000039F9FEF7E7FEFBF7F4FC0020FCF78CF822
:10491000FDF7CAFA2A4F7869400302D5FFF736FD42
:1049200018B30420FCF780F87869264D800414D46D
:10493000FFF7AAFDC8B1FFF7A7FDB0B1FFF7A4FDCF
:1049400098B10420FCF770F8A8681F497A699204AE
:1049500003D4AA68121A8A42F8D3A86842F21071E6
:10496000AA68121A8A42FBD36671FDF77DFAFBF73B
:104970004BFD80B100F07AF968B10220FCF754F8E1
:1049800094F90500401C03D110488069FFF744FFEB
:104990000120607004E00220FCF746F86670667142
:1049A000FFF7F4FC40B140210948FBF7DEFB402251
:1049B000D1010748FEF750FEFFF786FD0C000010FE
:1049C000008009200000094080841E00685100001A
:1049D00038010010F0B50B30154D20F00701002410
:1049E000144A0FE003688B420BD38B4205D95E1A41
:1049F00043184768C3E9006700E04368136002C0DA
:104A000004E0021D10680028ECD12046002802D1E5
:104A1000286808B10020F0BD064A07481060074A20
:104A2000121A22F00702C0E9002401202860D7E70B
:104A300034010010300100107C1D0010788D001032
:104A4000FFB50246002002EB420501464FF44056F6
:104A50006C4603AA6B1844F82130B34202DD0020F3
:104A600004B0F0BD094F07EB6307DB073F785754ED
:104A700001D03B095354535C8F0003F00F03535490
:104A8000BB40491C18440329E4DBE9E7910100100D
:104A9000084A32231360C2E9010107484FF47A71D2
:104AA0000068B0FBF1F0D06002F114011046FFF78E
:104AB00009BF00000C1C0010DC0000102DE9F047BD
:104AC0001D4A00234FF40077156A4FF4FF79C5F3B0
:104AD0000724DFF868A04FF4E05CDFF86480194E2B
:104AE00025E0B84216D213280CD014280CD0484523
:104AF0000CD0A0F58072FF3A0AD03E2813D81AF8DD
:104B0000002011E0EAB20FE022460DE055220BE052
:104B1000AA2209E0604506D208EB0002A2F5805205
:104B200092F8002E00E00022F254401C5B1C8B42E5
:104B3000D7D3BDE8F08700008C000010285100009A
:104B4000910100103801001070B50D462D494A69D9
:104B5000520302D5496D490521D4B0F5007F1ED31B
:104B6000294B2A4CB0F5E05F1AD29968A269891ADC
:104B7000274A914204D39968A16100216160616173
:104B8000244A0021A2F5D05307E044181C44565C87
:104B9000A4F58054491C84F8006EA942F5D370BD79
:104BA000616921B99968A16199686161A0601A4938
:104BB00049790029F3D199686269891A174A9142A3
:104BC0001BD2174A012111709968A161996861612E
:104BD000A168401A6168884203D9616A884200D29C
:104BE00060600620FBF720FF61682A46BDE8704040
:104BF000084801F50051FEF72FBDBDE870400C20BC
:104C0000FBF712BF00800920000009408C00001053
:104C1000A0860100911B00100C00001020A10700CD
:104C20007C000010FFB50DA60446E1CE8DE8E10042
:104C3000022902DA002004B0F0BD6018002100F85B
:104C4000011D6946B3FBF2F502FB1535B3FBF2F328
:104C50004D5D00F8015DA042F4D8ECE7303132330D
:104C600034353637383941424344454646F20440EC
:104C700000210088A0F51942993A0AD04FF4C040AB
:104C80004FF4002208C890421944FBD309B1002018
:104C9000704701207047000010B572B63324084BEE
:104CA00010C307C307484FF47A710068B0FBF1F0F6
:104CB0001860191D0248FFF705FE62B610BD00001E
:104CC0000C1C0010DC0000102DE9F041144C23688E
:104CD00003B920600020134D636803E00F5C1E18C9
:104CE000401CAF559042F9D398184FF4807660601D
:104CF000B04212D12068FFF79BFD0A4D143D286891
:104D000000B1FEE7324607492068FFF7C5FF286873
:104D100000B1FEE70020606020600020BDE8F08167
:104D2000C4000010341C001000050F0A1B1E1411D3
:104D300033363C39282D272263666C69787D77727B
:104D400050555F5A4B4E4441C3C6CCC9D8DDD7D26B
:104D5000F0F5FFFAEBEEE4E1A0A5AFAABBBEB4B15B
:104D600093969C99888D878283868C89989D97924B
:104D7000B0B5BFBAABAEA4A1E0E5EFEAFBFEF4F13B
:104D8000D3D6DCD9C8CDC7C240454F4A5B5E54512B
:104D900073767C79686D676223262C29383D37321B
:104DA00010151F1A0B0E040103060C09181D17120B
:104DB00030353F3A2B2E242160656F6A7B7E7471FB
:104DC00053565C59484D4742C0C5CFCADBDED4D1EB
:104DD000F3F6FCF9E8EDE7E2A3A6ACA9B8BDB7B2DB
:104DE00090959F9A8B8E848180858F8A9B9E9491CB
:104DF000B3B6BCB9A8ADA7A2E3E6ECE9F8FDF7F2BB
:104E0000D0D5DFDACBCEC4C143464C49585D5752AA
:104E100070757F7A6B6E646120252F2A3B3E34319A
:104E200013161C19080D07020000211042206330E0
:104E30008440A550C660E770088129914AA16BB1F2
:104E40008CC1ADD1CEE1EFF131121002733252229A
:104E5000B5529442F772D662399318837BB35AA342
:104E6000BDD39CC3FFF3DEE362244334200401146A
:104E7000E664C774A44485546AA54BB52885099592
:104E8000EEE5CFF5ACC58DD553367226111630063A
:104E9000D776F6669556B4465BB77AA719973887E2
:104EA000DFF7FEE79DD7BCC7C448E5588668A778FA
:104EB0004008611802282338CCC9EDD98EE9AFF932
:104EC000488969990AA92BB9F55AD44AB77A966ADA
:104ED000711A500A333A122AFDDBDCCBBFFB9EEB82
:104EE000799B588B3BBB1AABA66C877CE44CC55CAA
:104EF000222C033C600C411CAEED8FFDECCDCDDDD2
:104F00002AAD0BBD688D499D977EB66ED55EF44E79
:104F1000133E322E511E700E9FFFBEEFDDDFFCCF21
:104F20001BBF3AAF599F788F8891A981CAB1EBA175
:104F30000CD12DC14EF16FE18010A100C230E320F1
:104F40000450254046706760B9839893FBA3DAB399
:104F50003DC31CD37FE35EF3B1029012F322D23241
:104F60003542145277625672EAB5CBA5A895898569
:104F70006EF54FE52CD50DC5E234C324A014810491
:104F80006674476424540544DBA7FAB79987B89739
:104F90005FE77EF71DC73CD7D326F2369106B016E1
:104FA00057667676154634564CD96DC90EF92FE9F9
:104FB000C899E9898AB9ABA9445865480678276831
:104FC000C018E1088238A3287DCB5CDB3FEB1EFBD9
:104FD000F98BD89BBBAB9ABB754A545A376A167A81
:104FE000F10AD01AB32A923A2EFD0FED6CDD4DCDA9
:104FF000AABD8BADE89DC98D267C076C645C454CD1
:10500000A23C832CE01CC10C1FEF3EFF5DCF7CDF78
:105010009BAFBABFD98FF89F176E367E554E745E20
:10502000932EB23ED10EF01E005EBCE2613FDD83E6
:10503000C29C7E20A3FD1F419DC3217FFCA2401E78
:105040005F01E3BD3E6082DC237D9FC1421CFEA068
:10505000E1BF5D0380DE3C62BEE0025CDF81633D58
:105060007C22C09E1D43A1FF4618FAA427799BC548
:1050700084DA3866E5BB5907DB856739BAE4065838
:105080001947A5FB7826C49A653BD987045AB8E628
:10509000A7F91B45C6987A24F8A6441A99C7257B18
:1050A0003A6486D85B05E7B98CD2306EEDB3510F08
:1050B0004E10F2AC2F7193CD114FADF3702ECC92F8
:1050C000D38D6F31B2EC0E50AFF1134DCE90722CE8
:1050D0006D33D18F0C52B0EE326C8ED0530DEFB1D8
:1050E000F0AE4C1291CF2D73CA947628ABF51749C8
:1050F0000856B4EA6937D58B5709EBB536688AD4B8
:1051000095CB2977F4AA4816E9B7550B88D6346AA7
:105110002B7597C94A14F6A8742AC896154BA9F797
:10512000B6E80A54D7896B35EB3C904D53444F5346
:10513000352E3000020201000110000004F80C00BE
:10514000010001000000000000000000000029EF45
:10515000BEADDE41544F4C20465072696E744641DC
:105160005431322020200000000000000010000018
:10517000002000000030000000400000005000004F
:10518000006000000070000000800000009000003F
:1051900000A0000000B0000000C0000000D000002F
:1051A00000E0000000F000000000010000800100AD
:1051B00000000200008002000000030000800300E5
:1051C00000000400008004000000050000800500CD
:1051D00000000600008006000000070000800700B5
:1051E000FF0F0000FF1F0000FF2F0000FF3F000027
:1051F000FF4F0000FF5F0000FF6F0000FF7F000017
:10520000FF8F0000FF9F0000FFAF0000FFBF000006
:10521000FFCF0000FFDF0000FFEF0000FFFF0000F6
:10522000FF7F0100FFFF0100FF7F0200FFFF020080
:10523000FF7F0300FFFF0300FF7F0400FFFF040068
:10524000FF7F0500FFFF0500FF7F0600FFFF060050
:10525000FF7F0700FFFF0700120110010000004060
:1052600051C203130001042048010902200001017A
:10527000008032090400000208065062070582021D
:105280004000000705020240000000040309041C5E
:1052900003410054004F004C00200020002000205B
:1052A000002000200020002000200028034600509D
:1052B00000720069006E007400200046006C0061FE
:1052C0000073006800200020002000200020002043
:1052D0000020001A034600690072006D007700612B
:1052E000007200650030003000300030000E034DC9
:1052F0000065006D006F0072007900003D3A00000B
:1053000000000000713B00000000000000000000F1
:10531000000000000000000000000000000000008D
:10532000000000000000000000000000000000007D
:10533000000000000000000000000000E10200008A
:10534000E10200007D070000A10700007D070000CA
:10535000A1070000A1070000A107000059070000F5
:10536000E1020000E10200007D070000A10700004B
:105370007D070000A1070000A1070000A1070000B1
:1053800059070000F5220000ED220000192000005E
:10539000191F00005124000029280000452B00009F
:1053A0009D2B00003D210000F5030000F7020000E6
:1053B000D5120000191F0000512400005D170000E5
:1053C000053300006118000001140000432F0000A5
:1053D0003D2F000019200000191F0000512400007B
:1053E000492F0000053300005D3300003D2100001F
:1053F00000000000000000000000000000000000AD
:10540000000000000000000000000000000000009C
:1054100000000000345400000000001038010000BB
:10542000F80100006054000038010010409C0000AA
:105430007C4300000114BD41544F4C20465072691A
:105440006E74280548D4284B3D32130266102C0E8A
:10545000270780C3C90100879303044D6CDC020059
:105460004190313F689E67B6565C22364F4299BCE8
:10547000994F228F7F4D95CA2F14E8F2C63F55E60B
:105480007478F00FDDDA0346DC5ED10F4A9AECEE59
:1054900051EE8B1C947E9A56ED6A23893E66ED533D
:1054A00030810DC5CC15B241F92F9458999CF8550F
:1054B000D44ED053E9D13436AADABEFE3A35663737
:1054C000CB81D0165F4EE910A96C61CA147730C742
:1054D0002C6454C4A7DD4D9AE18CD0E77A7FF49711
:1054E00089D533D74EE216524B4D2CCF275715EAAC
:1054F000A31AD9CF0748D929D76E6A19F5411E1BBF
:1055000090D54B1199ACE1BD9AAE21305DD3896243
:105510006A1D54A9866F64789B4E7B43FCC66A263D
:1055200094E31941BB813419F334A31A64C7EE9292
:10553000DAE21C64BB1A550A88FDC736E56B4D914B
:105540001EE422FD7677DC7890366EF104C5DFB27A
:10555000BE5E574FAB55C13FFFDF320B5420EE8B81
:10556000022E6BE2F18B35ABFB7DEA6355E2A0F3D3
:10557000A478FF759B35D68E94184B9FB5A20E6507
:10558000B6AD11514BB5DA8D7C64DBCF6EB922D943
:1055900090CF030275A41DED4B8FADD943B2119589
:1055A00074A3A044DBF27069B209C7137C5594B0B0
:1055B0008070043EA8C3AA4F6D0521319532D1E019
:1055C000D2C04FA81EB7BDE087FF12271751B2689F
:1055D000F3ADF0C48F8E00DA245F6B2E92BAA82E42
:1055E000940FDEA75EB2D52E8321CED434A7945279
:1055F000AC0E8A290D842E800A1B7FCA9337CCD823
:10560000B25CF3D3E15ADD677704CC9EA0AF802D66
:1056100030FD8A6B379070D29AB6F56F959F6DD238
:10562000D3ACB06FF640865E62613C38F4E1BE58A0
:10563000808428391D9C5120E5A8A41E25C2DBAF1B
:10564000FCEB5D62973E0FD68D60394CEEC142692E
:10565000C228BE5A61A2B28870C25095FE03671874
:105660005B8E24A7BD0D96A7B67ED517E03F7D774C
:10567000E949A745EA5D5934F664FFECA08FA3140D
:10568000674E96A0FBD2397FF80D6709B98C543765
:105690008CE868058CB0E1BF3A91327BDF23330D93
:1056A00041A84BCF100E78A04E8763BD02530D1258
:1056B000C5620A4D15DA73032B5639B2F089434E91
:1056C0000FFE45A1B78A6E54EF6F1133508F99DEEC
:1056D000773B858515CD1B032C221B2D12A4A969B0
:1056E000F449DF3A939A87927FDFD6982185E800C4
:1056F000D16228B1C9BD758EFEB0CE9C271100A223
:10570000F7B4AA324CE39DEBE1530AF78D150C5820
:1057100033F888ABBD0E5623E43F240DC332A68E6A
:10572000EC283BE24E0A5817225BE405E867F43B9D
:105730002A285B5322B5391D318D480F90DAB16BA1
:10574000920D1A59DB27530989ECF703E503BB7760
:105750003CF9919B9AE93B3D8EBD905954B2ED7353
:10576000A78F53E47032E53DE2BF7BC4EF0C14EA2F
:1057700079E98FA5BEE4064BBBB257AD4776A0EEE4
:105780009D79C5A8CBB042CEC610E469D51FB62F0F
:10579000CB4508CF14DE4C0F11C30329C3566D341B
:1057A000F8E2C6258B7CD305FD6A0EEF3F682E2FED
:1057B00085C50F35DFA498A33494EB0F285EE20F64
:1057C0004C61142C81856546D660E34877259E5848
:1057D000AF331AABE79061FC6569EECB977F731A24
:1057E0003B455CC06C26E9E3367541934E0A38436D
:1057F0007B9655EBA0C0D4C16F637DC1C35C1E1FF7
:105800008DF4F996A84AFD572053046871F6E5DC3B
:105810002BFD5550EE91395DA53939610C0CC2E86C
:1058200095C8A2613687A4D71365B6EABB979E5B7D
:10583000BB1E6D877D43AA983897BA1FD5E715CE52
:10584000B238C11DD259CB095B6D30D6D86B92509E
:10585000A78B63877B68C083C3CAA52B46D465D357
:10586000DE26EDB3A541F0F8990722901F65561B7F
:1058700021BF8F9CA081564C6F1FFDB01B2B522C5B
:105880007545CFE7557C138441C6292A53B4AC73C0
:105890006AC6B8FE0AAAF245DA0622243095491AE9
:1058A000C4170FA83FDF9DFE2472443DBC0462C3B1
:1058B000CD0C74B57E3744CAF89432FE3F88171B6E
:1058C000A761EBAD8CC5132CE19B21251E68C2B9E5
:1058D000C25E7BF52721F61772A484A2057900C564
:1058E0002FBDDA14C5F1EC9818FE24FAF07E5C5B4B
:1058F00097DF75DD075B41DB7B21B44FF44E1E5211
:105900004CB4C622332B79DC11BF698E384260D685
:10591000D67A2A9F173E0DCDD30B9327D314E235A9
:10592000FA5256A9240BCB78B8224FE3E121AA2DD5
:1059300049999108D222BE053E137C0BD7CCE5AA2B
:10594000C6E60B8C42735AE90ACE12DD82A7478065
:1059500075544931EB6942E85190F5B86D8E8885F0
:105960002BE77239A21D6B99A3D56F268F2360DEBA
:10597000FD66842B261D30A7B1E924E003DD9A23C0
:10598000B14BE76D7DD401BB816D0F63B39B0D35CA
:10599000AE3CA970A3BD097E892623E640F9055FC8
:1059A00070E023F8A3401E64B4DA1726B41907A7E1
:1059B000FC48A02BC6810DD496D99BC24747807165
:1059C00085670DCEF44F3085F1735AD98B6B2F77E5
:1059D000420584EE0CD5EBDA0F97885448394768B6
:1059E0001BF2B168FF008C488716868AC48C10733E
:1059F000D587D7845C277B0B39DAC64B6A6B929AC2
:105A0000B89DB38AFA82348D4BCF5CDE8662B62AAB
:105A100023E2AB76A395DDE1E6ECCFB013800D0C6D
:105A200059334CA11E8E769F2A8C4EE94A58BB658D
:105A3000CF52400B765A3395A6A198862464B5932D
:105A4000629CE9348EF4F88F3E2336675017EC02DF
:105A5000FA449CF392C8FE3E5758B0AEB8422B832E
:105A6000CBB69E896E7DDB64D55FDEDFC716CC7A50
:105A7000DC68BDDECD0F0415EE0141F00FCED90379
:105A8000C2CF95677E2A8805FE855092FC13C7AF6A
:105A900024146B2A3BE9531D15B0807113FE2DDFD2
:105AA000F4BD680F8B423FD4D6500F2865EEB81B6B
:105AB0002F408090A9531621FB22808C383576F236
:105AC0000D6A61DE66C73B89C72F4BC282382A5AEE
:105AD0006FE2C41B2231C562EE25642BB4A0712D88
:105AE000A7679C12A1129C6862F9DEE9034E91EA55
:105AF0009A4D44B3D81924A20D504154B5092486B7
:105B0000E62BC477353A7A267A3802FF366A95FB57
:105B10004955D61F634F929F75A0E969EC8A1E9D77
:105B200000A76C79A068B12522428DBF02E418421B
:105B3000F3FEFB817584C64C857404256930A24749
:105B400022334E4B294821D7C70547A022E466459A
:105B5000B90CEC5CA94ABBCC03B1CE3866CF579EDA
:105B60005304B86540B08C9798CA20ACFF85E7AC69
:105B7000A8B17B2C9BC6D6FD3E02A9C3B8D442ED8A
:105B8000B681E275E23C8F6779579B3C220F39B3AF
:105B9000884BF0F7C3C69C001EB0D0AA633428DE41
:105BA00023DE6D00E3615F1772E80E86E58C752ECB
:105BB0003D2D0A42997B21B713DD05099CD712F0D0
:105BC0002829D01F345C1111E4318E9FD775F596CA
:105BD00062DFFF258BD01FAA06C0C324119D079545
:105BE00000DF1BD18C3D824254B6DB44893152D355
:105BF000A7CC910EB278DB9BACBA77D96797683E99
:105C00000BFF65652FB9296CFAEEF78116E89885C8
:105C100044EA3FB1914B239046730B15D2764DCD9C
:105C2000D759F3517E8CA483B4942C761059060274
:105C3000CD220906B9627D1DF1C546D4D86659B793
:105C4000ABEA501CB4FC62B59CAE658045A2604ACC
:105C500039A9866E68076A4C530F51C23AEE28E59F
:105C600091F3FCE4B46663502321E1699B4D35A1B7
:105C7000013D66BBEC06E457C20AC8F447224CDC7F
:105C800031C793EBC7AA7D1E7827F464C07D8EAD23
:105C9000C1BEF75A1E89CF014B2285818825840811
:105CA00005FA69F1D544FD200866E758C09DFC61FE
:105CB000D247A46B7F43254ECE72C4267740820A1A
:105CC00034133451B62C5925F9037CFA915AEC243B
:105CD000A379814B367B9F44FD066C30AB3D4A5A1D
:105CE0009FFDCB99C2A9544D5D574BBEFF5C88E424
:105CF0003806FE1D67CE462892B8B68AB511E61D55
:105D0000CD669E4E3D32F74017A0598B3773997878
:105D1000C0B4F154A9CBD6C87CFD26E5A7B07EF669
:105D2000B9F8F679B239F4E20D001C9D05BDD165D4
:105D3000A7A942AA3E0B945BC2CBBD7F092DBD6AC9
:105D400098829FB783A3D729727C15ADBBC8BBE7E8
:105D500053AE64980F00E76D55FD67D791309B8176
:105D6000BAC50BD9CC99DD1A3185F13946861003B5
:105D70003818C957E994D78BE54CD1B12DB39D960E
:105D80002D92E2A2342E4545FA54F9FE3533F1E066
:105D9000BBEF710A87D2F622719098539E9FB4F49C
:105DA000807A9B7748593FEBE83D51FF5DC07B41CE
:105DB000EBEF0132BFDB14CA402A42F95274CDE244
:105DC0000C672A8AD3E3EBD91084AD9AE6F7C16653
:105DD000E1F0E7E0B7D126A7CD77A75C6C6F1E1680
:105DE000698FA7DCB282EE89D57018403BDE4FED9B
:105DF00008D93628484B7B2B313E7B1A5E2FF5EABB
:105E00002D98F793A989DA85ADB5B018B8F19F0739
:105E10007678CA599103C6A77116444BFD937F1E2D
:105E2000EAF30F6FF75C9305045A64894ACD254C59
:105E3000420469949A09059C58C828BB3FFE472331
:105E400025773E7E2ED474F496188F61053A93E23E
:105E5000CF0073CC2F902474C83D063F9DB3F7E765
:105E60005F9E86A4E9BBB6E3CE3A3491BD850B3F75
:105E7000740945D2393E596905E5D0448CCC41A915
:105E8000C1A0C649C80C3709AFBB3FA5D605A1675D
:105E900013237289467B7B0ADE39E364BCE472CE4D
:105EA000390C71808DD536859A7CDCEC3E4C093DF1
:105EB000F7037FB13E0F13E4A5F542E6D165B8D9EB
:105EC0006D8950D57FA330095D4E2EEC197D386E5B
:105ED00013705E5E03AA80626F953D7DBC2106460D
:105EE0004BD85BD07BB71B1445DBC0954FCDD7118A
:105EF000128BC4B180D5F3D08C32DEC1C35A40F6C8
:105F0000EA7E35AF61B6AA77B34A3B3D355214B944
:105F10001D880D92EFF729B97A79C26978E9097A73
:105F20005B5E56C14CCBCBD1A03DBE3A082EC9EF2B
:105F3000CA6941021D8BF34404A6510E568026E423
:105F4000A907C415506FEA60DB8BB75DA74409DB76
:105F500019C3A8908E3AD0F1ADD602335A60E2D67A
:105F6000981AB8E63DDD353AA908E3D531755513E1
:105F7000A724E8B820864AF9962B89E4F9641854D6
:105F8000460CAC79D22EAD560BC48329E00D73D8E4
:105F900008EFF74D41FA5D067E25811F9E70267839
:105FA000679724EFF8C07570DED63510A7AA466D46
:105FB0000A0747364F16A4C5F2D72E96EBA687CA16
:105FC00007934C0CA89830DC5E1E57AE7D1868E82D
:105FD000D3992137E13ECFDDC99A9C253ADFB55BE5
:105FE0004D7BA0F4590A94A6BE6428259283C4F27E
:105FF000C34DE3C2DC1D2AD5DDF69DE0F4DB3CA9F0
:00000001FF
